:100000000C94E9000C9404010C9404010C94040178
:100010000C9404010C9404010C941E120C94040121
:100020000C9404010C9404010C9433170C94F416F2
:100030000C9449110C9404010C9404010C940401D7
:100040000C9404010C941F040C9404010C940A10E9
:100050000C945D100C9404010C9404010C940401A4
:100060000C9404010C9404010C9404010C940401FC
:100070004570692D4F5344205665722E302E382E10
:1000800031610000416B7475656C6C65732053655C
:100090007474696E67000053657474696E6720201C
:1000A0000000486F6568656E73656E736F7220003F
:1000B000004853206D697420536368616C746572E5
:1000C00020000048656164696E6720486F6C642099
:1000D00000004B6F6D706173732000004B6F6D708B
:1000E0006173732066697820000047505320416B8C
:1000F00074697620000041636873656E6B6F707081
:10010000656C756E67200000447265687261746585
:1001100020626567722E2000004665686C6572205B
:1001200046433C2D3E4F53442000004B65696E65AD
:100130002053657474696E672D416E7A65696765D1
:10014000000050432F4254206973742065696E6724
:1001500065736368616C7465740000DC6265726E5F
:1001600065686D65204C65747A7465732053657499
:1001700074696E6700004F4E00002D2D2D00004960
:10018000497D49491849497E49491949497B4949A5
:100190001D49497C49492149497D49491849497EB8
:1001A0004550492D4D656E750050616C0050432FD0
:1001B0004254004B656E6E756E670052432D42656A
:1001C0007472696562000045786974004F4E002DB5
:1001D0002D0011241FBECFEFD4E0DEBFCDBF11E054
:1001E000A0E0B1E0ECEBFFE202C005900D92AC3470
:1001F000B107D9F713E0ACE4B1E001C01D92A23819
:10020000B107E1F70C9411010C94000080E981BB67
:100210008FE084BBAC9AAD9A8EE28ABBD99ADD9A04
:1002200008951F93109294011092900110929501DD
:10023000A0E0B0E00E94CA17802D99278093530157
:10024000A1E0B0E00E94CA17802D99278093000199
:10025000A2E0B0E00E94CA17802D99278093540134
:10026000A7E1B0E00E94CA17802D9927809367010B
:10027000A8E1B0E00E94CA17802D992780937A01E7
:100280000E9499160E9406010E940E04809153015B
:10029000813019F40E94F50F02C00E94E50F789496
:1002A000A89A0E94A4030E9480040E9413090E943D
:1002B0008F090E941B0980914E018130F1F4109248
:1002C0004E0180919401882351F4809153019091C3
:1002D0005C01882321F4913011F40E94FF10809179
:1002E0007301813021F4109273010E9488120E94E0
:1002F0003C110E9441110E949514809152019091ED
:100300009401813041F4992331F40E947F0E0E94C0
:1003100020140E947C13809151018130C9F5809195
:1003200094018823A9F5AA9A0E94FD0E8091670185
:100330008823B9F40E94E5070E94D50680917A01CE
:1003400080FF04C00E94BC110E94EF090E943A087D
:100350000E943F0980917A0183FF19C00E94C20B5D
:1003600016C080910201823054F00E943A080E9427
:100370003F090E94BC110E94EF090E94C20B8091AC
:100380000201833024F00E94E5070E94D506AA9856
:1003900080914C018130B1F580919401882391F5D1
:1003A00010924C0180916701882321F08091020115
:1003B000833014F00E941B098091640190916501C3
:1003C00001969093650180936401809164019091FE
:1003D0006501CC9769F48091620190916301019667
:1003E0009093630180936201109265011092640101
:1003F0000E94240C0E947D0980915901813011F4E2
:100400000E94D80C10914D01113009F054CF809109
:100410009401882309F04FCF10924D018091800103
:10042000813019F0823059F406C00E94EA0982E056
:100430008093800104C00E94CD09109380018091B7
:100440006701813009F037CF80919401882309F04A
:1004500032CF80916601813009F02DCF1092660174
:1004600080910201813071F082301CF4882339F0D0
:1004700022CF823081F0833009F01DCF17C00E9457
:10048000EA0919CF0E94CD0964E084E00E945D0270
:100490000E94810410CF0E94CD0964E084E00E9494
:1004A0005D020E9413090E948F0905CF0E94CD09A9
:1004B00064E084E00E945D02F8CE482FD99827E0DE
:1004C00030E0DB98000000000000000081E090E0D8
:1004D000022E02C0880F991F0A94E2F7842311F0BC
:1004E000DA9A01C0DA980000000000000000DB9AF0
:1004F0000000000000000000215030408FEF2F3F2F
:100500003807F9F627E030E0DB9800000000000033
:10051000000081E090E0022E02C0880F991F0A942B
:10052000E2F7862311F0DA9A01C0DA9800000000A1
:1005300000000000DB9A00000000000000002150D5
:1005400030408FEF2F3F3807F9F6DB98DA98D99AC9
:10055000089564E084E00E945D026CE480E00E9403
:100560005D0210924E0180914E018823E1F36AE012
:100570008CE60E945D0260E085E00E945D020895C5
:100580001F93CF93DF9380914C018823E1F3109266
:100590004C010E94B11010E00DC0809151018130DA
:1005A00011F40E94FD0E80914C01813019F41092DB
:1005B0004C0111E090917B0180E0112309F481E06E
:1005C000992311F4882349F7C8E1D0E0882309F47E
:1005D000A4C080916D0380937A0180917A01DE013D
:1005E000082E0E94D21744E850E062E082E00E94A8
:1005F000660B47E950E064E082E00E94660B42EA45
:1006000050E066E082E00E94660B41EB50E067E05C
:1006100082E00E94660B43EC50E068E082E00E94BA
:10062000660B42ED50E069E082E00E94660B4CED03
:1006300050E06AE082E00E94660B4AEE50E06BE018
:1006400082E00E94660B46EF50E06CE082E00E9480
:10065000660B409178015091790164E084E10E9439
:100660003B0B80917A0180FF03C046E751E002C056
:100670004AE751E066E084E10E94660B80917A01CE
:1006800081FF03C046E751E002C04AE751E067E05E
:1006900084E10E94660B80917A0182FF03C046E7E5
:1006A00051E002C04AE751E068E084E10E94660B35
:1006B00080917A0183FF03C046E751E002C04AE718
:1006C00051E069E084E10E94660B80917A0184FF29
:1006D00003C046E751E002C04AE751E06AE084E126
:1006E0000E94660B80917A0185FF03C046E751E0C6
:1006F00002C04AE751E06BE084E10E94660B809102
:100700007A0186FF03C046E751E002C04AE751E0A4
:100710006CE084E10E94660B13C044E850E062E0A4
:1007200082E00E94660B49E151E065E082E00E94B0
:10073000660BDE010E94CA17802D992780937A01EB
:10074000DF91CF911F9108950E94A90210924C0150
:1007500080914C018823E1F340E750E062E087E0BC
:100760000E94660B0E94810410924C0180914C0102
:100770008823E1F310924C0180914C018823E1F32E
:1007800010924C0164E084E00E945D026CE480E021
:100790000E945D0280915301882319F40E94C002D7
:1007A0001AC04BE251E062E082E00E94660B42E434
:1007B00051E064E082E00E94660B4BE551E066E0A8
:1007C00082E00E94660BA8E1B0E00E94CA17802D6B
:1007D000992780937A0180914C018823E1F310924C
:1007E0004C0180914C018823E1F310924C018091DF
:1007F0004C018823E1F310924C0180914C01882335
:10080000E1F310924C0180914C018823E1F31092A6
:100810004C0164E084E00E945D02089582E083BFA1
:1008200082E48EBD8EE189BF83E087BD86E982BD0B
:1008300083E480938A0080E280937D0008951F9274
:100840000F920FB60F9211248F939F9380915001B6
:100850008F5F8093500180915001883439F591E089
:1008600090934F011092500180917A038F5F809393
:100870007A0380917A03843631F410927A0390934C
:100880004C0190934D0180917A03823311F490933F
:100890004D01809179038F5F809379038091790373
:1008A0008A3021F41092790390934E019F918F9199
:1008B0000F900FBE0F901F901895282F80538A30ED
:1008C00010F090E005C0203311F49AE001C0982F99
:1008D000822F81548A3110F4922F9653822F8156A1
:1008E0008A3110F4922F9C532D3211F499E403C0F5
:1008F0002E3209F491E4892F992787FD9095089568
:10090000089560E085E00E945D0263E886E00E9451
:100910005D0260E987E00E945D0260E085E00E9480
:100920005D0264E886E00E945D0261E987E00E9462
:100930005D0260E085E00E945D0265E886E00E945D
:100940005D0262E987E00E945D0260E085E00E944E
:100950005D0266E886E00E945D0263E987E00E942E
:100960005D0260E085E00E945D0267E886E00E942B
:100970005D0264E987E00E945D0260E085E00E941C
:100980005D0268E886E00E945D0265E987E00E94FA
:100990005D0260E085E00E945D0269E886E00E94F9
:1009A0005D0266E987E00E945D0260E085E00E94EA
:1009B0005D026AE886E00E945D0267E987E00E94C6
:1009C0005D0260E085E00E945D0261EA86E00E94CF
:1009D0005D0268E987E00E945D0260E085E00E94B8
:1009E0005D0262EA86E00E945D0269E987E00E949A
:1009F0005D0260E085E00E945D0263EA86E00E949D
:100A00005D026AE987E00E945D0260E085E00E9485
:100A10005D0264EA86E00E945D026BE987E00E9465
:100A20005D0260E085E00E945D0265EA86E00E946A
:100A30005D026CE987E00E945D0260E085E00E9453
:100A40005D0266EA86E00E945D026DE987E00E9431
:100A50005D0260E085E00E945D0267EA86E00E9438
:100A60005D026EE987E00E945D0260E085E00E9421
:100A70005D0268EA86E00E945D026FE987E00E94FD
:100A80005D0260E085E00E945D026FEB86E00E94FF
:100A90005D0260EA87E00E945D0260E085E00E94FE
:100AA0005D0260EC86E00E945D0261EA87E00E94E0
:100AB0005D0260E085E00E945D0261EC86E00E94DC
:100AC0005D0262EA87E00E945D0260E085E00E94CC
:100AD0005D0262EC86E00E945D0263EA87E00E94AC
:100AE0005D0260E085E00E945D0263EC86E00E94AA
:100AF0005D0264EA87E00E945D0260E085E00E949A
:100B00005D0264EC86E00E945D0265EA87E00E9477
:100B10005D0260E085E00E945D0265EC86E00E9477
:100B20005D0266EA87E00E945D0260E085E00E9467
:100B30005D0266EC86E00E945D0267EA87E00E9443
:100B40005D0260E085E00E945D026DED86E00E943E
:100B50005D0268EA87E00E945D0260E085E00E9435
:100B60005D026EED86E00E945D0269EA87E00E9408
:100B70005D0260E085E00E945D026FED86E00E940C
:100B80005D026AEA87E00E945D0260E085E00E9403
:100B90005D0260EE86E00E945D026BEA87E00E94E3
:100BA0005D0260E085E00E945D0261EE86E00E94E9
:100BB0005D026CEA87E00E945D0260E085E00E94D1
:100BC0005D0262EE86E00E945D026DEA87E00E94AF
:100BD0005D0260E085E00E945D0263EE86E00E94B7
:100BE0005D026EEA87E00E945D0260E085E00E949F
:100BF0005D0264EE86E00E945D026FEA87E00E947B
:100C00005D0260E085E00E945D026BEF86E00E947D
:100C10005D0260EB87E00E945D0260E085E00E947B
:100C20005D026CEF86E00E945D0261EB87E00E944E
:100C30005D0260E085E00E945D026DEF86E00E944B
:100C40005D0262EB87E00E945D0260E085E00E9449
:100C50005D026EEF86E00E945D0263EB87E00E941A
:100C60005D0260E085E00E945D026FEF86E00E9419
:100C70005D0264EB87E00E945D0261E085E00E9416
:100C80005D0260E086E00E945D0265EB87E00E9405
:100C90005D0261E085E00E945D0261E086E00E9405
:100CA0005D0266EB87E00E945D020895FF920F935C
:100CB0001F93CF93DF938C01F62EEC0117C06D2F9D
:100CC000772785E00E945D026C2F86E00E945D021E
:100CD0008F2D9927FC01EE0FFF1FE80FF91FE15F31
:100CE000FE4F608187E00E945D022196C801059653
:100CF000C817D90720F3E8012A9617C06D2F772768
:100D000085E00E945D026C2F86E00E945D028F2DBF
:100D10009927FC01EE0FFF1FE80FF91FE15FFE4F5F
:100D2000608187E00E945D022196C8010F96C81776
:100D3000D90720F3DF91CF911F910F91FF90089574
:100D40000F931F93CF93DF938C01EC010EC06D2F97
:100D5000772785E00E945D026C2F86E00E945D028D
:100D600060E087E00E945D022196C8010596C817E1
:100D7000D90768F3E8012A960EC06D2F772785E022
:100D80000E945D026C2F86E00E945D0260E087E0B9
:100D90000E945D022196C8010F96C817D90768F313
:100DA000DF91CF911F910F9108951F93CF93DF9300
:100DB000809121039091220366E170E00E94B717B1
:100DC0009B012E5F3F4F37FD1BC0C9016AE070E0F9
:100DD0000E94B717182F1695C9016AE070E00E94AB
:100DE000B71787E090E0861B91092EE130E0829FE3
:100DF000E001839FD00D929FD00D1124279616C03D
:100E0000309521953F4FC9016AE070E00E94B71705
:100E1000182F16951C5FC9016AE070E00E94B71791
:100E20008EE1689FE0011124C950DF4F80910B01D2
:100E300090910C01C817D90739F080910B0190915E
:100E40000C010E94A00604C080917E01811721F050
:100E5000612FCE010E94560610937E01D0930C01A3
:100E6000C0930B01DF91CF911F910895AF92BF9274
:100E7000DF92EF92FF920F931F93CF93DF93CDB743
:100E8000DEB721970FB6F894DEBF0FBECDBF8C0141
:100E9000D62E5C0119826B2D772785E00E945D02BA
:100EA0006A2D86E00E945D02ED2CFF24F701E35DD0
:100EB000FE4F608187E00E945D028EE190E0A80E07
:100EC000B91E9981925E99839C3329F7F4EBAF2E7A
:100ED000B12CA00EB11E6B2D772785E00E945D021C
:100EE0006A2D86E00E945D02F701E35DFE4F60819E
:100EF00087E00E945D02EEE1F0E0AE0EBF1EC80189
:100F0000825F9E4FA816B90631F721960FB6F89466
:100F1000DEBF0FBECDBFDF91CF911F910F91FF902C
:100F2000EF90DF90BF90AF900895EF92FF920F93F4
:100F30001F93CF93DF93CDB7DEB721970FB6F89409
:100F4000DEBF0FBECDBF8C017C0119826F2D7727CC
:100F500085E00E945D026E2D86E00E945D0260E0E9
:100F600087E00E945D028EE190E0E80EF91E998113
:100F7000925E99839C3351F784EBE82EF12CE00EBE
:100F8000F11E6F2D772785E00E945D026E2D86E0B1
:100F90000E945D0260E087E00E945D02EEE1F0E009
:100FA000EE0EFF1EC801825F9E4FE816F90649F754
:100FB00021960FB6F894DEBF0FBECDBFDF91CF9163
:100FC0001F910F91FF90EF9008951F93CF93DF93A0
:100FD000809123039091240366E170E00E94B7178B
:100FE0009B012A5F3F4F37FD12C0C9016AE070E0E4
:100FF0000E94B717182F16951C5FC9016AE070E0B0
:101000000E94B717C6E8D0E0C61BD10913C03095BF
:1010100021953F4FC9016AE070E00E94B717182F71
:101020001695C9016AE070E00E94B717C62FDD2748
:10103000C957DF4F80910D0190910E01C817D90754
:1010400039F080910D0190910E010E94950704C026
:1010500080917F01811721F0612FCE010E94360718
:1010600010937F01D0930E01C0930D01DF91CF91BA
:101070001F910895FF920F931F93CF93DF93809159
:101080003303909134038E55904063E070E00E94EA
:10109000B717EB016A3071051CF0C9E0D0E004C05D
:1010A00077FF02C0C0E0D0E08091600190916101C3
:1010B000C817D90709F47DC0C230D10514F468E11E
:1010C00001C068E084E00E945D02D0936101C0939A
:1010D0006001C530D105B9F1C630D1057CF4C2300C
:1010E000D10521F1C330D1051CF42197A9F419C011
:1010F000C330D10501F1249779F421C0C730D1055F
:1011000049F1C730D1051CF1C830D10531F129971B
:1011100019F4BBE8FB2E23C0A8E8FA2E04E810E877
:1011200020C0F8E8FF2E04E811E81BC0E8E8FE2E16
:1011300004E812E816C078E8F72E04E811C068E861
:10114000F62E05E80DC058E8F52E06E809C048E877
:10115000F42E05C039E8F32E02C02AE8F22E07E883
:1011600013E860E085E00E945D026FE186E00E9486
:101170005D02612F87E00E945D0260E085E00E94D1
:101180005D026DE386E00E945D02602F87E00E94B1
:101190005D0260E085E00E945D026BE586E00E94F2
:1011A0005D026F2D87E00E945D0260E084E00E9496
:1011B0005D02DF91CF911F910F91FF900895EF9203
:1011C000FF920F931F93CF93DF937A019EE1699F64
:1011D000B0011124680F711D8B01020F111D1092B7
:1011E0007B03EB0116C06D2F772785E00E945D021F
:1011F0006C2F86E00E945D0280917B03F701E80F6F
:10120000F11D60818F5F80937B0387E00E945D0208
:101210002196C017D10738F3DF91CF911F910F911D
:10122000FF90EF90089525E046E051E06EE081E008
:101230000E94DF080895CF93DF93CDB7DEB72597DF
:101240000FB6F894DEBF0FBECDBFDE011196EAE304
:10125000F1E085E001900D928150E1F725E0AE01CB
:101260004F5F5F4F67E08CE00E94DF0825960FB666
:10127000F894DEBF0FBECDBFDF91CF910895CF931D
:10128000DF93CDB7DEB724970FB6F894DEBF0FBE5D
:10129000CDBF19821A8285E48B831C82309133037F
:1012A000832F6AE00E949717282F0E949717482FD4
:1012B000822F0E949717292F832F0E949717992317
:1012C00019F48AE08C8301C09C83222319F48AE0FC
:1012D0008A8301C02A83498324E0AE014F5F5F4FB8
:1012E00062E083E00E94DF0824960FB6F894DEBF28
:1012F0000FBECDBFDF91CF91089580915401813011
:1013000069F420919A01922F27FD9F5F95954BE9F3
:1013100051E061E08EE0891B0E94DF08089560E0E3
:1013200085E00E945D026FE186E00E945D0260E858
:1013300087E00E945D0260E085E00E945D026DE34F
:1013400086E00E945D0264E887E00E945D0260E042
:1013500085E00E945D026BE586E00E945D0268E820
:1013600087E00E945D02089560E085E00E945D02D2
:101370006FEC86E00E945D026CE887E00E945D02EF
:1013800061E085E00E945D026BE086E00E945D0204
:101390006DE887E00E945D0208956CE480E00E94A1
:1013A0005D0208958091350390913603843B910549
:1013B00044F480918001882361F481E0809380016E
:1013C000089580918001181614F40E94CD0910929E
:1013D0008001089562E480E00E945D020895EF922A
:1013E000FF920F931F93CF93DF93CDB7DEB72F9765
:1013F0000FB6F894DEBF0FBECDBF85E0FE01369676
:1014000011928A95E9F780912B0390912C036EE15C
:1014100070E00E94B717CB018E01055F1F4F019747
:1014200097FF02C080E090E04AE050E0B8010E94DF
:101430006617F80101900020E9F73197EE2EE01AC7
:1014400010927B03FF240AC00E0F1F1FEC0FFD1F1D
:1014500083850E945D04F8018083F394EF2DFF27BC
:101460008E2D992787FD90958E010F5F1F4FE817EE
:10147000F90754F3F0927B0325E0AE014A5F5F4F1A
:1014800069E085E10E94DF082E2DA80169E089E16D
:101490008E190E94DF082F960FB6F894DEBF0FBE9C
:1014A000CDBFDF91CF911F910F91FF90EF900895E5
:1014B000EF92FF920F931F93CF93DF93CDB7DEB7D9
:1014C0002E970FB6F894DEBF0FBECDBF19821A82D9
:1014D0001B821C8280917001909171018E01065FC8
:1014E0001F4F4AE050E0B8010E946617F8010190D2
:1014F0000020E9F73197EE2EE01A10927B03FF24CB
:101500000AC00E0F1F1FEC0FFD1F82850E945D0495
:10151000F8018083F394EF2DFF278E2D992787FD07
:1015200090958E010B5F1F4FE817F90754F3F09267
:101530007B0324E0AE014F5F5F4F66E085E10E94D0
:10154000DF082E2DA80166E089E18E190E94DF08D0
:1015500080917001909171011816190664F460E091
:1015600085E00E945D0262EC86E00E945D026CE80C
:1015700087E00E945D02809170019091710197FF58
:101580000CC060E085E00E945D0262EC86E00E9493
:101590005D026DE887E00E945D028091700190918C
:1015A0007101892B61F460E085E00E945D0262ECCC
:1015B00086E00E945D0260E087E00E945D022E9658
:1015C0000FB6F894DEBF0FBECDBFDF91CF911F9154
:1015D0000F91FF90EF9008959F92AF92BF92CF929C
:1015E000DF92EF92FF920F931F93CF93DF93CDB7CC
:1015F000DEB76E970FB6F894DEBF0FBECDBF982E44
:10160000A62E7A01FA0101900020E9F73197BE2E4B
:10161000B41ACC24DD240BC0FF278A010E0F1F1F34
:10162000EE0DFF1D80810E945D04F8018083EC2D8A
:101630000894C11CD11C8B2D99270196AE014F5FD8
:101640005F4FC816D90641F72B2D6A2D892D0E94B0
:10165000DF086E960FB6F894DEBF0FBECDBFDF91E8
:10166000CF911F910F91FF90EF90DF90CF90BF909F
:10167000AF909F900895EF92FF920F931F93CF9397
:10168000DF93CDB7DEB764970FB6F894DEBF0FBE19
:10169000CDBFE82EF62ECA014AE050E08E010F5F62
:1016A0001F4FB8010E946617A8016F2D8E2D0E9452
:1016B000EC0A64960FB6F894DEBF0FBECDBFDF9183
:1016C000CF911F910F91FF90EF900895BF92CF920D
:1016D000DF92EF92FF920F931F93CF93DF93CDB7DB
:1016E000DEB764970FB6F894DEBF0FBECDBFB82E3D
:1016F000C62E9A01DE01119605C0EA0FFB1F9083EA
:101700002F5F3F4F822F841BF9019491E82FFF2711
:10171000992399F7EA0FFB1F1082FD010190002029
:10172000E9F73197DE2EDA1AEE24FF2409C08D0185
:10173000020F111DF80180810E945D04F801808371
:101740002E2D0894E11CF11C8D2D99270196DE01A8
:101750001196E816F90659F72D2DAD016C2D8B2D3C
:101760000E94DF0864960FB6F894DEBF0FBECDBFAF
:10177000DF91CF911F910F91FF90EF90DF90CF906D
:10178000BF900895EF92FF920F931F93CF93DF9333
:10179000CDB7DEB72B970FB6F894DEBF0FBECDBF27
:1017A000DE011196E7E3F1E083E001900D928150B4
:1017B000E1F78E01085F1F4F4AE050E0B8018091C9
:1017C0003103909132030E946617F80101900020C6
:1017D000E9F73197EE2EE01A10927B03FF240AC03E
:1017E0000E0F1F1FEC0FFD1F80850E945D04F80186
:1017F0008083F394EF2DFF278E2D992787FD9095F9
:101800008E010C5F1F4FE817F90754F3F0927B032A
:1018100023E0AE014F5F5F4F6EE08DE00E94DF0876
:101820002E2DA8016EE080E18E190E94DF082B9614
:101830000FB6F894DEBF0FBECDBFDF91CF911F91E1
:101840000F91FF90EF900895EF92FF920F931F93E7
:10185000CF93DF93CDB7DEB728970FB6F894DEBFEE
:101860000FBECDBF19828AE08A8380916201909178
:1018700063018E010A5F1F4F4AE050E0B8010E94E9
:101880006617F80101900020E9F73197EE2EE01A73
:1018900010927B03FF240DC08E010D5F1F4F0E0FB2
:1018A0001F1FEC0FFD1F86810E945D04F8018083DD
:1018B000F394EF2DFF278E2D992787FD9095E8173C
:1018C000F90754F3F0927B038091620190916301D8
:1018D0008E010D5F1F4F0A976CF421E0AE014F5F40
:1018E0005F4F6EE081E00E94DF0821E0A8016EE01A
:1018F00082E004C022E0A8016EE081E00E94DF08DF
:1019000080916401909165018E010A5F1F4F4AE04A
:1019100050E0B8010E946617F80101900020E9F735
:101920003197EE2EE01A10927B03FF240DC08E013A
:101930000D5F1F4F0E0F1F1FEC0FFD1F86810E94B2
:101940005D04F8018083F394EF2DFF278E2D9927F6
:1019500087FD9095E817F90754F3F0927B03809187
:101960006401909165018E010D5F1F4F0A976CF421
:1019700021E0AE014E5F5F4F6EE084E00E94DF0821
:1019800021E0A8016EE085E004C022E0A8016EE03D
:1019900084E00E94DF0828960FB6F894DEBF0FBEE1
:1019A000CDBFDF91CF911F910F91FF90EF900895E0
:1019B000CF92DF92EF92FF920F931F93CF93DF931B
:1019C000CDB7DEB72B970FB6F894DEBF0FBECDBFF5
:1019D00080915A0190915B0162E070E00E94B7171C
:1019E00070935B0160935A0180915A0190915B0161
:1019F0008456904090935B0180935A0180915A01E4
:101A000090915B0197FF04C010925B0110925A0104
:101A100080915A0190915B018D5A964234F08CEA84
:101A200096E290935B0180935A0180915A019091C4
:101A30005B0164E670E00E94A31770935601609307
:101A4000550180915A0190915B0164E670E00E941B
:101A5000A31790935801809357018091570190915B
:101A600058016AE070E00E94A317709358016093D8
:101A70005701809155019091560125E429831A82DE
:101A80001B828E01085F1F4F4AE050E0B8010E94A0
:101A90006617F80101900020E9F73197CE2EC01AA1
:101AA00010927B03DD240BC0020F131FE20EF31E06
:101AB000F70180810E945D04F8018083D3942D2D6D
:101AC00033278C2D992787FD909548E0E42EF12C43
:101AD000EC0EFD1E8E010C5F1F4F2817390724F3F3
:101AE000D0927B0322E0AE014E5F5F4F63E083E064
:101AF0000E94DF082C2DA80163E085E08C190E946C
:101B0000DF0880915701909158014AE050E0B701F9
:101B10000E946617F70101900020E9F73197EE194E
:101B2000EE2E10927B03FF240AC00E0F1F1FEC0F36
:101B3000FD1F80850E945D04F8018083F394EF2DE2
:101B4000FF278E2D992787FD90958E010C5F1F4FE3
:101B5000E817F90754F3F0927B0321E0AE014F5FE1
:101B60005F4F63E085E00E94DF0821E0AE014E5F39
:101B70005F4F63E086E00E94DF0821E0A80163E098
:101B800086E00E94DF082B960FB6F894DEBF0FBEEA
:101B9000CDBFDF91CF911F910F91FF90EF90DF901C
:101BA000CF9008950F931F93CF93DF93CDB7DEB7F8
:101BB0002A970FB6F894DEBF0FBECDBF4AE050E0C3
:101BC0008E010F5F1F4FB8010E946617F801019048
:101BD0000020E9F73197E01B10927B0320E0FF27FC
:101BE000E7FDF09501C02F5F822F99278E179F0781
:101BF000D4F320937B032A960FB6F894DEBF0FBE72
:101C0000CDBFDF91CF911F910F910895EF92FF9279
:101C10000F931F93CF93DF9333E0E32EF12CC0E0BB
:101C2000D0E0ACE8B2E08C91FD012181128103810A
:101C3000B7016C5F7F4F7B011496F2E0673C7F0732
:101C400009F456C0422F55274D535040E0914301AF
:101C5000F0914401EC0FFD1F9927CD97880F991F34
:101C6000880F991F9A01689413F835952795169453
:101C7000E1F7822B932B80836B317105C9F1212F02
:101C800033272D533040FE013196809143019091CE
:101C90004401E80FF91F4F70507084E0440F551F46
:101CA0008A95E1F7C9019595879595958795482B74
:101CB000592B408381E06F367807D1F0FE013296D0
:101CC0008091430190914401E80FF91F2370307017
:101CD00086E0220F331F8A95E1F7802F9927CD9751
:101CE000282B392B2083635C724011F023969BCF05
:101CF000DF91CF911F910F91FF90EF900895EF9298
:101D0000FF920F931F93CF93DF938091B10184349F
:101D100009F06AC033E0E32EF12C60E070E0A2EB42
:101D2000B1E08C91FD01218112810381E7012496AC
:101D30007E0114966134710509F456C0422F55276F
:101D40004D535040E0914101F0914201E60FF71FE1
:101D50009927CD97880F991F880F991F9A0168942A
:101D600013F8359527951694E1F7822B932B8083F2
:101D700060347105C9F1212F33272D533040FB0109
:101D800031968091410190914201E80FF91F4F7007
:101D9000507084E0440F551F8A95E1F7C90195956D
:101DA000879595958795482B592B4083CB35D10541
:101DB000D9F0FB0132968091410190914201E80FE8
:101DC000F91F2370307046E0220F331F4A95E1F768
:101DD000802F9927CD97282B392B20836E337105BF
:101DE00019F06D5F7F4F9DCF10925201DF91CF911F
:101DF0001F910F91FF90EF900895EF92FF920F9334
:101E00001F93CF93DF9380918B02843409F089C0B4
:101E100033E0E32EF12C60E070E0ACE8B2E08C91AE
:101E2000FD01218112810381E70124967E01149630
:101E30006134710509F456C0422F55274D53504067
:101E4000E0913F01F0914001E60FF71F9927CD97F0
:101E5000880F991F880F991F9A01689413F8359578
:101E600027951694E1F7822B932B808360347105BC
:101E7000C9F1212F33272D533040FB01319680913A
:101E80003F0190914001E80FF91F4F70507084E0BE
:101E9000440F551F8A95E1F7C9019595879595954A
:101EA0008795482B592B4083CB35D105D9F0FB01C1
:101EB000329680913F0190914001E80FF91F237005
:101EC000307046E0220F331F4A95E1F7802F9927A3
:101ED000CD97282B392B20836E33710519F06D5F58
:101EE0007F4F9DCF8091350390913603843B9105C0
:101EF0006CF410925C01F8940E94F50F7894809134
:101F0000350390913603843B91055CF080915C0130
:101F1000882339F481E080935C01F8940E94E50FF6
:101F2000789480918B028C3459F481E090E0909306
:101F300079018093780181E080937B010E94060EF5
:101F400080918B028D3459F482E090E09093790176
:101F50008093780181E080937B010E94060E80913E
:101F60008B028E3459F483E090E090937901809352
:101F7000780181E080937B010E94060E80918B02A4
:101F80008F3459F484E090E0909379018093780144
:101F900081E080937B010E94060E80918B02803548
:101FA00059F485E090E0909379018093780181E085
:101FB00080937B010E94060E10925101DF91CF9118
:101FC0001F910F91FF90EF90089582E289B910BCA4
:101FD00080B91CBE909A28E92AB996E890BD82EC97
:101FE0008BB921B99CBF82B9089582E289B910BC2E
:101FF00080B91CBE909A88E98AB926E820BD92EC87
:102000009BB980E981B92CBF92B90895159BFECF89
:1020100083B908951F920F920FB60F9211248F93D8
:102020009F93EF93FF939CB190937C039D3081F439
:1020300080918201813061F4AB981092820180938B
:102040005201E0916403FF27E155FE4F90832CC0BD
:1020500080918201882319F0813031F513C09332C9
:1020600039F480915201882319F481E08093820130
:102070001092640380916403E82FFF27E155FE4F1F
:1020800090830CC0E0916403FF27E155FE4F9083DD
:1020900080916403853930F4809164038F5F80936D
:1020A000640302C010928201FF91EF919F918F9182
:1020B0000F900FBE0F901F9018951F920F920FB6A2
:1020C0000F9211248F939F93EF93FF9393B190936B
:1020D0007D039D3081F480918101813061F4AB9862
:1020E0001092810180935101E0916103FF27E7572E
:1020F000FD4F90832DC080918101882319F081309C
:1021000039F514C0933241F480915101882321F4B0
:1021100081E080938101AB9A109261038091610309
:10212000E82FFF27E757FD4F90830CC0E091610334
:10213000FF27E757FD4F908380916103853930F485
:10214000809161038F5F8093610302C010928101CF
:10215000FF91EF919F918F910F900FBE0F901F9065
:102160001895CF93DF93CDB7DEB72C970FB6F894C1
:10217000DEBF0FBECDBF83E289831A8281E78B83E6
:102180008CE78C838DE68D838DE38E838F8320E0B7
:1021900030E0FE013196AE01485F5F4F8191280F1C
:1021A000311DE417F507D1F7C90160E070E10E9425
:1021B000B7179C0160E470E00E94B717635C688702
:1021C000C90160E470E00E94B717835C89878DE0E5
:1021D0008A87FE0131969E01255F3F4F8081159BC6
:1021E000FECF83B93196E217F307C1F72C960FB6ED
:1021F000F894DEBF0FBECDBFDF91CF910895CF938E
:10220000DF93CDB7DEB72A970FB6F894DEBF0FBEC7
:10221000CDBF83E289831A8283E68B831C821D8271
:1022200086E890E060E070E10E94B7179C0160E4EE
:1022300070E00E94B717635C6E83C90160E470E0D0
:102240000E94B717835C8F838DE08887FE013196EB
:102250009E01275F3F4F8081159BFECF83B931964A
:10226000E217F307C1F72A960FB6F894DEBF0FBE48
:10227000CDBFDF91CF91089585B392E0892785BBCB
:10228000089590915F01913019F485B3892785BB3A
:1022900008951F920F920FB60F9211242F933F9320
:1022A0005F936F937F938F939F93AF93BF9380912F
:1022B000830190918401892B81F484B595B5909325
:1022C0008A01809389018EB58F7B8EBD81E090E07D
:1022D000909384018093830141C084B595B5909318
:1022E0008801809387012EB520642EBD209189013D
:1022F00030918A01821B930B10928401109283010A
:10230000865698406CE271E00E94A3177093860194
:102310006093850177FF05C01092860110928501B8
:1023200009C06730710534F086E090E09093860133
:102330008093850120918501309186018091020171
:10234000992787FD90952817390741F026303105E8
:102350002CF42093020181E080936601BF91AF913C
:102360009F918F917F916F915F913F912F910F90EE
:102370000FBE0F901F90189580912B0390912C0306
:10238000909369018093680180916801909169013F
:1023900020916A0130916B01821B930B90936D0128
:1023A00080936C01809168019091690190936B0119
:1023B00080936A01409174015091750120916C01E4
:1023C00030916D01CA01E3E0880F991FEA95E1F7AA
:1023D000841B950B73E0220F331F7A95E1F7820F70
:1023E000931F68E070E00E94B717709375016093C7
:1023F00074012091760130917701409174015091E0
:102400007501C90163E0880F991F6A95E1F7821B86
:10241000930B840F951F68E070E00E94B7177093CC
:102420007701609376018091760190917701909386
:102430007101809370010E94580A08951F920F92B3
:102440000FB60F9211242F933F935F936F937F9357
:102450008F939F93AF93BF9380918B01882391F4C7
:10246000809180009091810090938D0180938C01E8
:1024700080918A008F7B80938A0081E080938B011A
:10248000949A38C010928900109288008091800040
:102490009091810020918A00206420938A001092FC
:1024A0008B01949820918C0130918D01821B930BAC
:1024B0008A5F904090938F0180938E0169E170E074
:1024C0000E94A3177093880260938702809187020D
:1024D000909188028856914030F087E691E0909381
:1024E000880280938702809187029091880281E020
:1024F00080937301BF91AF919F918F917F916F9165
:102500005F913F912F910F900FBE0F901F901895E4
:10251000CF93DF93CDB7DEB760970FB6F894DEBFE9
:102520000FBECDBF80918702909188026FE070E06E
:102530000E94A317AE014B5F5F4FDA01641BCE010F
:102540004096E62FEA0FFF27E158FE4FE491ED9306
:10255000A817B907B1F719821A821B821C822BE0D7
:102560006BE089E00E94DF0824E0AE014F5F5F4F1F
:102570006CE08EE00E94DF08409187025091880253
:102580006CE08FE00E943B0B60960FB6F894DEBFC4
:102590000FBECDBFDF91CF910895BF92CF92DF9252
:1025A000EF92FF920F931F93CF93DF93CDB7DEB7D8
:1025B00060970FB6F894DEBF0FBECDBF19821A82A6
:1025C0001B821C8280917D0290917E0290938103F8
:1025D0008093800380917F029091800290937F038B
:1025E00080937E0380918003909181038E01055F2B
:1025F0001F4F4AE050E0B8010E946617F8010190B1
:102600000020E9F73197BE2EB01ACC24DD240DC08E
:10261000EC0CFD1CF70180810E945D040C0D1D1D5A
:10262000F80180830894C11CD11C8B2D992787FD4C
:1026300090952BE0E22EF12CEC0EFD1E8E010B5F2F
:102640001F4FC816D90624F324E0AE014F5F5F4F39
:1026500061E08CE00E94DF082B2DA80161E080E1A1
:102660008B190E94DF0880917E0390917F034AE0DE
:1026700050E0B7010E946617F70101900020E9F7CA
:102680003197DE2EDE18EE24FF240DC0FE01EE0D84
:10269000FF1D83850E945D040E0D1F1DF8018083C0
:1026A0000894E11CF11C8D2D992787FD90958E01D2
:1026B0000B5F1F4FE816F9064CF324E0AE014F5FA5
:1026C0005F4F62E08CE00E94DF082D2DA80162E0E0
:1026D00080E18D190E94DF0860960FB6F894DEBF86
:1026E0000FBECDBFDF91CF911F910F91FF90EF9063
:1026F000DF90CF90BF9008958F929F92BF92CF921C
:10270000DF92EF92FF920F931F93CF93DF93CDB79A
:10271000DEB760970FB6F894DEBF0FBECDBF19824B
:102720001A821B821C8280904503909046038E0182
:10273000055F1F4F4AE050E0B8018091430390913C
:1027400044030E946617F80101900020E9F73197D1
:10275000BE2EB01ACC24DD240DC0EC0CFD1CF701FC
:1027600080810E945D040C0D1D1DF801808308947A
:10277000C11CD11C8B2D992787FD90953BE0E32E42
:10278000F12CEC0EFD1E8E010B5F1F4FC816D906F3
:1027900024F324E0AE014F5F5F4F64E08CE00E94C1
:1027A000DF082B2DA80164E080E18B190E94DF086F
:1027B0004AE050E0B701C4010E946617F70101909A
:1027C0000020E9F73197DE2EDE18EE24FF240DC03D
:1027D000FE01EE0DFF1D83850E945D040E0D1F1D81
:1027E000F80180830894E11CF11C8D2D992787FD49
:1027F00090958E010B5F1F4FE816F9064CF324E00D
:10280000AE014F5F5F4F65E08CE00E94DF082D2D29
:10281000A80165E080E18D190E94DF0860960FB67F
:10282000F894DEBF0FBECDBFDF91CF911F910F9106
:10283000FF90EF90DF90CF90BF909F908F90089582
:10284000DF92EF92FF920F931F93CF93DF93CDB759
:10285000DEB72B970FB6F894DEBF0FBECDBFDE01FB
:102860001196E9E4F1E083E001900D928150E1F7E7
:102870008E01085F1F4F4AE050E0B8018091850249
:10288000909186020E946617F80101900020E9F7F6
:102890003197DE2ED01AEE24FF240DC0FE01EE0D7E
:1028A000FF1D80850E945D040E0D1F1DF8018083B1
:1028B0000894E11CF11C8D2D992787FD90958E01C0
:1028C0000C5F1F4FE816F9064CF323E0AE014F5F93
:1028D0005F4F61E088E10E94DF082D2DA80161E0D3
:1028E0008BE18D190E94DF082B960FB6F894DEBF9E
:1028F0000FBECDBFDF91CF911F910F91FF90EF9051
:10290000DF90089522E047E451E061E08AE10E940F
:10291000DF080895F89488E190E028E00FB6F89475
:10292000A89581BD0FBE21BDFFCF1F939D9902C108
:10293000809190018F5F8093900191E0909392013C
:1029400080919001853009F0F9C08091940188232D
:1029500009F071C0909394011092950164E084E0B5
:102960000E945D0220919A014BE951E061E083E011
:102970000E94DF0840EA51E063E083E00E94660BBA
:1029800068E084E00E945D0249EA51E065E083E08E
:102990000E94660B80910001813019F44CEC51E0EB
:1029A00002C04FEC51E065E084E10E94660B60E0FC
:1029B00084E00E945D024DEA51E066E083E00E94FF
:1029C000660B80915301813019F44CEC51E002C048
:1029D0004FEC51E066E084E10E94660B43EB51E06E
:1029E00067E083E00E94660B80915401813019F406
:1029F0004CEC51E002C04FEC51E067E084E10E94F2
:102A0000660B4BEB51E068E083E00E94660B80911F
:102A10006701813019F44CEC51E002C04FEC51E0F9
:102A200068E084E10E94660B47EC51E06BE083E0D4
:102A30000E94660B81C010919501113001F568E08C
:102A400084E00E945D0280915301882329F4109351
:102A500053014CEC51E004C0109253014FEC51E093
:102A600066E084E10E94660B80915301A0E0B0E033
:102A7000082E0E94D21760E084E00E945D028091DF
:102A80009501823009F568E084E00E945D02809142
:102A90005401882331F481E0809354014CEC51E0DF
:102AA00004C0109254014FEC51E067E084E10E94B1
:102AB000660B80915401A2E0B0E0082E0E94D2176C
:102AC00060E084E00E945D0280919501833009F509
:102AD00068E084E00E945D0280916701882331F400
:102AE00081E0809367014CEC51E004C010926701D3
:102AF0004FEC51E068E084E10E94660B8091670131
:102B0000A7E1B0E0082E0E94D21760E084E00E94A6
:102B10005D0280919501843089F410929401F894BB
:102B200088E190E028E00FB6F894A89581BD0FBE2B
:102B300021BDFFCF10929001109292019C99E9C0A3
:102B400090919401913009F0EAC0909393018091A3
:102B500091018F5F8093910180919101853009F0FF
:102B6000DEC01092910180919501823009F464C019
:102B7000833030F4882359F0813009F0D0C031C05F
:102B8000833009F483C0843009F0C9C09EC090939B
:102B9000950149EA51E065E083E00E94660B80916F
:102BA0000001813019F44CEC51E002C04FEC51E0CF
:102BB00065E084E10E94660B68E084E00E945D02AB
:102BC0004DEA51E066E083E00E94660B809153017C
:102BD000813019F44CEC51E002C04FEC51E066E05A
:102BE00090C082E0809395014DEA51E066E083E079
:102BF0000E94660B80915301813019F44CEC51E036
:102C000002C04FEC51E066E084E10E94660B68E090
:102C100084E00E945D0243EB51E067E083E00E94A4
:102C2000660B80915401813019F44CEC51E002C0E4
:102C30004FEC51E067E065C083E08093950143EB82
:102C400051E067E00E94660B80915401813019F4D5
:102C50004CEC51E002C04FEC51E067E084E10E948F
:102C6000660B68E084E00E945D024BEB51E068E097
:102C700083E00E94660B80916701813019F44CEC6F
:102C800051E002C04FEC51E068E03BC084E080932B
:102C900095014BEB51E068E083E00E94660B809168
:102CA0006701813019F44CEC51E002C04FEC51E067
:102CB00068E084E10E94660B68E084E00E945D02A7
:102CC00047EC51E06BE083E01DC01092950147ECAA
:102CD00051E06BE083E00E94660B68E084E00E94B4
:102CE0005D0249EA51E065E083E00E94660B809155
:102CF0000001813019F44CEC51E002C04FEC51E07E
:102D000065E084E10E94660B60E084E00E945D0261
:102D100006C01092910180919201809193011F91C0
:102D20000895813029F4A0E0B0E0062E0E94D21769
:102D30000895EF92FF920F931F93CF93DF93CDB738
:102D4000DEB764970FB6F894DEBF0FBECDBF40E08C
:102D500050E08E010F5F1F4F842F9927DC01AD5F7C
:102D6000BF4F0E94CA17202D3327F801E80FF91F23
:102D700020832223F1F04F5F5F4F2F3F69F71082CE
:102D800018C0FE01E00FF11F81810E945D0405560D
:102D90001E4FF80180830E2D11270894E11CF11CB1
:102DA00080919A01992787FD9095081719074CF390
:102DB0000EC0DE011196FD0101900020E9F7319768
:102DC000EA1BFB0BE0939A01EE24FF24E4CF649608
:102DD0000FB6F894DEBF0FBECDBFDF91CF911F912C
:102DE0000F91FF90EF9008951F920F920FB60F92E0
:102DF00011248F939F93809199018130A1F08130AC
:102E000018F0823049F525C0809197018E3129F460
:102E10001092970181E080939901809197018F5FD3
:102E20008093970119C090919801923061F41092AB
:102E3000980180919601813019F49093990103C013
:102E400083E080939901809198018F5F809398012E
:102E500003C083E0809399019F918F910F900FBEE3
:102E60000F901F9018951F920F920FB60F9211247A
:102E70008F9380919901833011F4109299018F9171
:102E80000F900FBE0F901F90189580912103909185
:102E9000220365E070E00E94B71766507F4F77FD10
:102EA0000FC081E0653F78071CF064EF71E003C05C
:102EB0006B3F71053CF06A5F81E08093960104C02E
:102EC00060E070E01092960162BD0895FB019F01E1
:102ED000E8944230C4F04532B4F44A3029F497FB08
:102EE0001EF4909581959F4F642F77270E94A3171A
:102EF000805D8A330CF0895D8193CB010097A1F747
:102F000016F45DE251931082C9010C948717DC011D
:102F1000FC0101900020E9F73297AE17BF0730F4AB
:102F20007C916081708331976D93F7CF0895991BE1
:102F300079E004C0991F961708F0961B881F7A95B0
:102F4000C9F780950895AA1BBB1B51E107C0AA1FB2
:102F5000BB1FA617B70710F0A61BB70B881F991F3A
:102F60005A95A9F780959095BC01CD01089597FBDE
:102F7000092E07260AD077FD04D0E5DF06D0002011
:102F80001AF4709561957F4F0895F6F790958195A5
:102F90009F4F0895E199FECFBFBBAEBBE09A11965B
:102FA0000DB20895E199FECFBFBBAEBB0DBA11962D
:0C2FB0000FB6F894E29AE19A0FBE089563
:102FBC0001010200000A0000440000230023005419
:102FCC00646653636552620051610050600050604A
:102FDC00005161005262005363655464666768690E
:102FEC006A6B6B6A69686700000053536353531F25
:0C2FFC0003450265030D0A0A1D000000D9
:00000001FF
